:100000000C945C000C946E000C946E000C946E00CA
:100010000C946E000C946E000C946E000C946E00A8
:100020000C946E000C946E000C946E000C946E0098
:100030000C946E000C946E000C946E000C946E0088
:100040000C9495000C946E000C946E000C946E0051
:100050000C946E000C946E000C946E000C946E0068
:100060000C946E000C946E0000000007000201006A
:100070000003040600000000000000000102040864
:100080001020408001020408102001020408102002
:10009000040404040404040402020202020203032E
:1000A0000303030300000000250028002B000000CC
:1000B0000000240027002A0011241FBECFEFD8E043
:1000C000DEBFCDBF11E0A0E0B1E001C01D92A930BC
:1000D000B107E1F70E94FB010C9408020C940000A8
:1000E00061E083E00E948C0161E082E00E948C016B
:1000F00061E083E00E94C50161E082E00E94C501E9
:1001000068EE73E080E090E00E94020160E083E02E
:100110000E94C50168EB7BE080E090E00E94020154
:1001200061E083E00C94C50108951F920F920FB611
:100130000F9211242F933F938F939F93AF93BF936D
:100140008091010190910201A0910301B0910401FD
:100150003091000123E0230F2D3720F40196A11DDB
:10016000B11D05C026E8230F0296A11DB11D2093E5
:1001700000018093010190930201A0930301B093C9
:1001800004018091050190910601A0910701B091B1
:1001900008010196A11DB11D8093050190930601F0
:1001A000A0930701B0930801BF91AF919F918F91E8
:1001B0003F912F910F900FBE0F901F9018953FB752
:1001C000F8948091050190910601A0910701B091EA
:1001D000080126B5A89B05C02F3F19F00196A11D67
:1001E000B11D3FBF6627782F892F9A2F620F711D8F
:1001F000811D911D42E0660F771F881F991F4A9548
:10020000D1F70895CF92DF92EF92FF92CF93DF93D1
:100210006B017C010E94DF00EB01C114D104E104F9
:10022000F10479F00E94DF006C1B7D0B683E734087
:10023000A0F381E0C81AD108E108F108C851DC4FE9
:10024000ECCFDF91CF91FF90EF90DF90CF900895AA
:10025000789484B5826084BD84B5816084BD85B5A1
:10026000826085BD85B5816085BDEEE6F0E0808168
:1002700081608083E1E8F0E0108280818260808389
:10028000808181608083E0E8F0E08081816080830C
:10029000E1EBF0E0808184608083E0EBF0E080813E
:1002A00081608083EAE7F0E08081846080838081E0
:1002B0008260808380818160808380818068808388
:1002C0001092C1000895833081F028F4813099F0B4
:1002D0008230A1F008958630A9F08730B9F08430DB
:1002E000D1F4809180008F7D03C0809180008F7752
:1002F00080938000089584B58F7702C084B58F7D88
:1003000084BD08958091B0008F7703C08091B000C4
:100310008F7D8093B0000895CF93DF9390E0FC0130
:10032000E458FF4F2491FC01E057FF4F849188234C
:1003300049F190E0880F991FFC01E255FF4FA5910C
:10034000B4918C559F4FFC01C591D4919FB7611119
:1003500008C0F8948C91209582238C938881822305
:100360000AC0623051F4F8948C91322F3095832377
:100370008C938881822B888304C0F8948C91822B83
:100380008C939FBFDF91CF9108950F931F93CF93CD
:10039000DF931F92CDB7DEB7282F30E0F901E8597F
:1003A000FF4F8491F901E458FF4F1491F901E05790
:1003B000FF4F04910023C9F0882321F069830E9434
:1003C00063016981E02FF0E0EE0FFF1FEC55FF4F56
:1003D000A591B4919FB7F8948C91611103C01095C9
:1003E000812301C0812B8C939FBF0F90DF91CF9110
:1003F0001F910F9108950E9428010E947000C0E093
:10040000D0E00E9494002097E1F30E940000F9CF11
:04041000F894FFCF8E
:00000001FF
